:030000000219FDE5
:03000B000200A848
:03002B0002019738
:03005B000203415C
:030073000203275E
:1000800002030406080C10182030406080040608A3
:100090000C10182030406080A0C000070F1F3F05E3
:1000A000050D050305030302C2AF306308C2638573
:1000B0007C8AD2AF32C0D0C0E0206227E525600242
:1000C000E473E525F4C3334009758A00D263F57CF7
:1000D00001D4F58A758B00758D00D262D0E0D0D046
:1000E000D2AF32C3E526334009758A00D263F57C6E
:1000F00001F4F58AC262E526F4603B3068032072A1
:1001000013758B00758D00D0E0D0D0C292C295C21D
:1001100096D2AF32C292C295C296206E0C2066096A
:10012000740AD5E0FDE57E4290758B00758D00D098
:10013000E0D0D0D2AF32758A00D263757C00C28D18
:10014000D262212901C2306805206602D29201C222
:10015000306805206602D29501C23068052066022B
:10016000D29601C2C29330680A2066077408D5E0AF
:10017000FDD29201C2C29430680A2066077408D585
:10018000E0FDD29501C2C29730680A206607740864
:10019000D5E0FDD29601C2C2AFC2AD53E6EFC0D0EA
:1001A000C0E0D2D3D2AFE57D6009E57A6005757A0B
:1001B0000041D4757A01C2CEE52A60072074491542
:1001C0002A41087800790020742EE580307E01F401
:1001D00030E50278FF53DACF207E0343DA20307E09
:1001E0000343DA10C2D8C271E580307E01F430E5F5
:1001F0000279FFC3E89970CB306103752A18207427
:1002000003752A18885FD27020740DE52B600415E1
:100210002B411843DA01C2D8207002417AA85F202E
:100220006102C270207431C3E894F0400374F0F8A6
:10023000E8C4540F28F87984B703024158C313C3A4
:10024000138721200802C313200A06C3C898F84167
:100250005828F8500374FFF8C3E895685003E56820
:10026000F88822E52D54066011E533C313C3132427
:10027000062522F52250037522FF852224A824C3D7
:10028000E52495644002A8648825E569700241BEB2
:10029000C3E8AA699A5003E8FAE4F9EAC333FBE534
:1002A0006BF45B29400D256AF8E56A6002156A4027
:1002B0000B41BE0AC3E56A9A5002056A78FF882698
:1002C000C26EC3E52694F84002D26EC3E525944081
:1002D0004002D26420CF0AD0E0D0D043E610D2ADA5
:1002E00032C2CF053AE57D6009E57B6005757B008C
:1002F000611D757B017801E52A6005307402152ABD
:10030000C3E55F94014005756200611D756300756A
:100310006C00E5622401F56250037562FFD0E0D005
:10032000D043E610D2AD32C2AFC0D053E67FC26038
:10033000759100855694855795759104D0D0D2AFAC
:1003400032C2AF53E6EFC2ADC0D0C0E0C0F0D2D3EE
:10035000D2AFA8FBA9FCE57D6007C3E913F9E81358
:10036000F8C2D830710261B353DACF207E0343DA8A
:1003700010307E0343DA20D271E580307E01F42014
:10038000E502618A88278928A1E053DACF207E031D
:1003900043DA20307E0343DA10C2D8C271307402CF
:1003A000A1CC7800E580307E01F430E502A1CC8854
:1003B0005FA1B453DACF207E0343DA20307E0343BB
:1003C000DA10C271206102818C53DACF207E0343A0
:1003D000DA10307E0343DA20C2D8D271885A895BA2
:1003E000C3E89558F8E99559F97B007E087A00C36F
:1003F000E8948CE994005005755E00817E88217830
:10040000A2E6A8216055C3E894C8E994005008E426
:10041000D2E4FB7A0A8159C3E89468E99401500850
:10042000E4D2E3FB7A0F8159C3E894D0E9940250F7
:1004300008E4D2E2FB7A1E8159C3E894A0E994054E
:100440005008E4D2E1FB7A3C8159C3E89498E994DE
:10045000085008E4D2E0FB7A787E00C3E8955CFCA3
:10046000E9955DFD30E70AECF42401FCEDF434007D
:0E047000FD755E00C3EC9AED9E5003755E01B3
:10047E00885C895D855A58855B597802A1B4C3E8BA
:10048E009527F8E99528F9307C02A198307B02A1D6
:10049E0098307A02A19120750281AFE9FDE8FC81C6
:1004AE00CEE9C313F9E813F8307902A191E9C31329
:1004BE00F9E813F8307802A191E9C313FDE813FCB3
:1004CE0020612CC3EC941CED9402400281E5ED708A
:1004DE001EC3EC94C850180529E52970021529C3CE
:1004EE00E529940A5002A1CC755F00D270A1CCE52B
:1004FE0029600215297888E6F97400207F0878961D
:10050E00B90302789EE624FAFEE43400FFC3EC9EA3
:10051E00FCED9FFD9208B90310A208500720760942
:10052E00D276A137307602C276A2085016B9030DE4
:10053E00ECF42401FCEDF43400FD02055178007951
:10054E0000A198B90315EC33FCED33FDC3EC940A0E
:10055E00FCED9400FD50047C007D00C3EC94FFED97
:10056E009400400678FF7900A198EC8575F0A4C53B
:10057E00F0A2F733F8790040030205B478FF790052
:10058E000205B4E9C313F9E813F8307C0EE96002F2
:10059E0078FFC3E81338F8E43400F9C3E894FFE9B0
:1005AE009400400278FF885FD270206102A1CC7463
:1005BE001FF4552F4BF52FC274EB7002D274752AAF
:1005CE0018307403752A0A306102A1E020740353B7
:1005DE00DAFE207403752B06D0F0D0E0D0D0D2AD69
:1005EE0043E6103279010206107903020610790AE9
:1005FE00020610791E020610796402061079C802EE
:10060E0006107817E4D5E0FDD8FAD9F6227A147BD5
:10061E00780206377A107B8C0206377A0D7BB4028D
:10062E0006377A0B7BC80206377902B27DE4C29494
:10063E00D5E0FDD295D5E0FDC295D5E0FDD294D59D
:10064E00E0FDD292E576D5E0FDC2927496D5E0FD3E
:10065E00D9D9EAF8D5E0FDD8FBDBCEC29422C37C13
:10066E00007D0075F00005F0EA33FAEB33FB50F62F
:10067E00EB13FBEA13FAC3E9FFE8FEE89AF8E99BED
:10068E00F95004EFF9EEF8B3EC33FCED33FDD5F091
:10069E00DFEDF9ECF822E889F08A20D2D4F8A9F03F
:1006AE007B0030F70B7BFFF42401F8E9F43400F9FA
:1006BE00E88520F0A4ADF0F8E98520F0A4AFF0FEB7
:1006CE00ED2EF974003FFA7C04C3EA13FAE913F92C
:1006DE00E813F8DCF48BF030F70AE8F42401F8E9BB
:1006EE00F43400F9E889F0C2D4F8A9F02222C3E567
:1006FE004113F9E54013F8C3E54598F8E54699F935
:10070E00500CC3E89480E994FF4016020733C3E807
:10071E00947FE994005003020733787F7900020733
:10072E0033788079FF884A894B22E54A2547F8E5D8
:10073E004B3548F9854B20E4300701F43549FA3042
:10074E00E709C3EA94F04015020771C3EA940F500B
:10075E000302077178FF79FF7A0F0207717800792B
:10076E00007AF0C3E5249564500AC37401952450B1
:10077E000B02078FE54B20E70E02078FE54B30E7A4
:10078E0006884789488A492278A4E6FAC3E54A339F
:10079E00F8E54B33F9D1A4E930E70BC3E89480E9CF
:1007AE0094FF4013E1C9C3E8947FE994005002E13D
:1007BE00C9787F7900E1C9788079FFE820E715C311
:1007CE00E52398F84009C3E8940140030207F07846
:1007DE00010207F0E8F424012523F840030207F094
:1007EE0078FF884C2278A5E6FAA848A949D1A4E951
:1007FE0030E70CC3E89401E994FF4016020824C3C5
:10080E00E894FFE99400500302082478FF7900026F
:10081E000824780179FFE920E715C3E54C98F840E4
:10082E0009C3E89401400302084B780102084BE823
:10083E00F42401254CF8400302084B78FF8824224B
:10084E0078FFC26420693D206A12D264C3E54194E8
:10085E000A4009C3E52594405002C26479A1E760BD
:0E086E0023E541601F74FF8541F0848539F059
:10087C00306A0375F005A4F8C5F0600278FFC3E890
:10088C0095675002A867886622C3E54094C8E54185
:10089C009400E56650031401A6046002F56622027A
:1008AC0008AE2275E890227883E6FFE5E820ECF7A5
:1008BC00A8BDA9BE0573C3E57394084052757300B7
:1008CC00E9FA79A0E76044EA7007E574601B020856
:1008DC00E9C3E895746010E5745006600C140208C6
:1008EC00F50460F90208F5E574F574C39472401BC5
:1008FC007564C0C394044013756480C39404400BA6
:10090C00756440C39404400375640075BB0922E50B
:10091C0064F460020564E573B4070375BB102274BC
:10092C003279A687F0A4C5F0A2F733F8C3E8956432
:10093C004002A86488228824882588268867227526
:10094C0040007541F022C2AF75C820A8CCA9CDAA31
:10095C003A30CF010A75C824D2AFC3EA13FAE913AF
:10096C00F9E813F8AB3BAC3C883B893CC3E89BF8FB
:10097C00E99C20690A547FF9306702417521D2AD98
:10098C003D8A3DF9EA9D547FFA600478FF79FFAE09
:10099C003EAF3F8B3E8C3FC3EC9FFCC3E99CF542C2
:1009AC00A83BA93CC3E89EF8E99FF9C3E54113FBBA
:1009BC00E54013FAE82AF540E93BF541500675404D
:1009CC00FF7541FF411CAA40AB41AC40AD417E04D8
:1009DC007F02C3EB940440021E1FC3EB9408400239
:1009EC001E1FC3ED13FDEC13FCDEF7C3EA9CFAEB00
:1009FC009DFBEF6009C3E913F9E813F8DFF7EA2868
:100A0C00FAEB39FB8A408B4150067BFF8B408B41C4
:100A1C00C3EB94025002D2673069047F03414778DC
:100A2C0092E6FFC3E537948240110FC3E53794A0DB
:100A3C0040010FC3EF940640027F057E02E541C4DE
:100A4C00540FF9E541C454F0F8E540C4540F28F8AC
:100A5C00C3E89EFAE99400FB4009C3EA9402EB94C4
:100A6C000050047A02E4FB41C1AA40AB41EBC4FE46
:100A7C00EAC4540F4EFCC3EA9CFAEB9400FBC3E8A7
:100A8C0013C313F8EA28FAEB3400FB8A408B41C3FA
:100A9C00EB94024002C2677802EBC4FE7B00EAC40E
:100AAC00540F4EFAC3EA98FA4005C3940250027AE6
:100ABC00027892E6FF30600241C185525685535749
:100ACC00D26043E680C3E49AF8E49BF9C3E833F8B8
:100ADC00E933F93067026162E8FAE9FBD3E913FD07
:100AEC00E813FC88528953C3EF94036038EF20E07D
:100AFC000DE82CF8E93DF9ECFAEDFB020B1DE828AA
:100B0C00F8E939F9C3E82402F8E93400F97AFE7BF4
:100B1C00FFC3EF9403400E8A548B55884E894F8C3B
:100B2C00508D516196885489558A4E8B4F8C508DBF
:100B3C0051306920C3E53394034019E542A2E71311
:100B4C00F8E555F4240138400B20E7087554FFF400
:100B5C002401F5556196E8FAD3E813FC8852C3EFEB
:100B6C0094036020EF20E007E82CF8ECFA6182E8AF
:100B7C00282402F87AFEC3EF940340088A54884E66
:100B8C008C50619688548A4E8C50E56BC33350025E
:100B9C00646BF56B30600261A0753404D26043E67F
:100BAC0080E52D5406601FA840A941C2AF53E67FD3
:100BBC00759100C3E498F594E499F595759104D278
:100BCC006043E680D2AF22D26575440075200030B8
:100BDC006B03752040020BF2D26575440075204002
:100BEC00306B03752000D2AF7801206722E52D54BD
:100BFC00066002C265C3E541940540137802940572
:100C0C0040087803940540027806306902780A207F
:100C1C006019E544601530690AC3E5339403400359
:100C2C00D53406D2AFD26C81D471A8D2AF0000C239
:100C3C00AF20672AE541C3FB940F40027B0FEB24E6
:100C4C000530730123306A02742820620123F930C5
:100C5C0069027982E58D13E58B13C39940B1054484
:0F0C6C00E59B5440B5200281BE30690A08C3E8F9
:100C7B00940A400108811B20650261F2C26553E6AC
:100C8B007F7591003067107594007595FC75910414
:100C9B00D26043E68061F2AE40AF41C3EE33FEEF6C
:100CAB0033FF50047EFF7FFFC3E49EF594E49FF572
:100CBB00958198C3E5339402500261F2306502616D
:100CCB00F2D80281D2811BC26C53E67F75910085ED
:100CDB005494855595759104854E56854F57D26022
:100CEB0043E680D2AFE52D54066008206A02053337
:100CFB00020D0E306C0D206B0A20650715811581D6
:100D0B0002159A2278003064053065027801E537C8
:100D1B0075F007A4F9E5F028F5F0E9A2F013A2F1BC
:100D2B0013A2F213F537C394785003753778C3E5E4
:100D3B003795384008D266C292C295C2963060028F
:100D4B00A148855056855157D26043E68022207DBD
:100D5B0011C2AF754302C294D293D2AF759F80027A
:100D6B000F28C2AF754302C294D297D2AF759F8042
:100D7B00020F28307243207D20C2AF7543039001D0
:100D8B0075757E10C296C297306204D295A19CD223
:100D9B0094D2AF759F89020F28C2AF7543039001A0
:100DAB0075757E10C292C293306204D295A1BCD2EB
:100DBB0094D2AF759F81020F28207D17C2AF754368
:100DCB0003900150C296306202D295D2AF759F89C3
:100DDB00020F28C2AF754303900150C292306202DA
:100DEB00D295D2AF759F81020F28207D11C2AF75AE
:100DFB004304C293D297D2AF759F81020F28C2AF23
:100E0B00754304C297D293D2AF759F89020F2830D6
:100E1B007243207D20C2AF754305900164757E0837
:100E2B00C295C294306204D292C138D293D2AF75BC
:100E3B009F80020F28C2AF754305900186757E8097
:100E4B00C295C294306204D296C158D297D2AF7574
:100E5B009F80020F28207D17C2AF75430590014676
:100E6B00C295306202D292D2AF759F80020F28C218
:100E7B00AF75430590015AC2953062EBD296D2AF53
:100E8B00759F80020F28207D11C2AF754306C29754
:100E9B00D294D2AF759F89020F28C2AF754306C299
:100EAB0093D294D2AF759F81020F28307242207D6E
:100EBB0020C2AF754301900186757E80C292C293AA
:100ECB00306204D296C1D4D297D2AF759F81020FF4
:100EDB0028C2AF754301900164757E08C296C29714
:100EEB00306204D292C1F4D293D2AF759F89E128BC
:100EFB00207D16C2AF75430190015AC29230620237
:100F0B00D296D2AF759F81E128C2AF754301900194
:100F1B0046C296306202D292D2AF759F89C26622C8
:100F2B00900144757E00C292C295C296C293C29440
:100F3B00C297C26222788076FF0876FF0876FF0898
:100F4B0076FF087603087604087609087603087698
:100F5B0001087601788C76010876FF0876FF087613
:100F6B00FF0876FF0876FF0876030876FF0876FF02
:100F7B000876FF0876250876D00876FA0876FA0800
:100F8B0076040876FF08760108760008767A0876EC
:100F9B00FF08760108760108760008760322788729
:100FAB00E6FFC272BF0302D2727888E6C394036075
:100FBB0008C27DE630E102D27DC27E7889E630E15F
:100FCB0002D27EC3EF94026008758E01D273020FBA
:100FDB00E1758E00C273227880E6149000809378BE
:100FEB00A4F67881E6149000809378A5F67886E6CF
:100FFB001490008D9378A6F6789CE67538FF7539BA
:10100B000CB402067538A075390AB403067538821C
:10101B0075390578A3E61490009A93F569120F2B96
:10102B0022227896E6FA7897E6FB7888E6B40305F1
:10103B00C3EB940EFB307F047A007BFFC3EB9AFC6F
:10104B00C3948250027C827575000575EC8575F032
:10105B00A4C3E5F0947D40F222D27F112D1206013C
:0F106B007A007B007C101205F7E55F2AFA74000B
:10107A003BFBDCF37C04C3EB13FBEA13FADCF7FE5D
:10108A00C27F112D22E5EF20E6037520000520908E
:10109A003FFFE520146006901FFF14600093046070
:1010AA000375EF1253D9BF7581C043FF801205F251
:1010BA0075EF0243B203E5B3240420E70DF521E5F9
:1010CA00E320E0068521B343E301120F2B7580FF6D
:1010DA0075A40075F1F075D4DF75900275A5FC75DD
:1010EA00F2FD75D50275A61075A0FF75F3F175E2CC
:1010FA0041E4F8F6D8FD756B01120F401215E57838
:10110A00988676753001C2AF12060B12061B1206BC
:10111A00011206221206011206291206011216FEF1
:10112A0012060B12060B120606C2AF78FA79FA30CB
:10113A008507D9FBD8F7021C00120FA9120FE2117A
:10114A002C112D78988676120F2B75A90075B6800A
:10115A00757D0075885075891275C8247591047556
:10116A00D84075A82275B80275E690759B80759D62
:10117A000075D10E75BCC075BB0975BA1175E880CA
:10118A001205F2D2AF1208AB53DACF207E0343DA4C
:10119A0020307E0343DA1043DA01C2D8C271120644
:1011AA000BD2617B037A0CE55E70077A0CDB0302D3
:1011BA001133120601207003021133C270E55FC3B6
:1011CA00940240E1E52F541F856160F561B560D551
:1011DA00DAD5C26153DACF207E0343DA20307E03A8
:1011EA0043DA10C2D8C27178A2E67008D274E52F29
:1011FA0054E0F52FC275752900120606307409C32A
:10120A00E529940A4002D2751205F7780230740271
:10121A007800C3E55F9840F0C2AF12061B12061BA6
:10122A0012061BD2AF12060B754D007888E6B4037E
:10123A000261131205F7788CE6C394015003021376
:10124A0013E530C394015003021313207435C3E528
:10125A005F94FF5003021313C2AF120630D2AF12CB
:10126A000606C3E55F940150EFC2AF12061B1205D2
:10127A00FC12061BD2AF120606C3E55F94FF40E9D3
:10128A000217837F05D27F112D120606C2AFC27FD5
:10129A00112DAE5FC3E55F947FD2AF40761205F29F
:1012AA00C2AF120630D2AFDFDC1164C3EE94057808
:1012BA0097F612060B1216271217067F0AD27F110B
:1012CA002D120606C2AFC27F112DAE5FC3E55F9431
:1012DA007FD2AF50E61205F2C2AF12061B1205FC0E
:1012EA0012061BD2AFDFD61164EE24057896F612E9
:1012FA00060B121627121735120606112DC3E55FC3
:10130A0094FF50024155021783C3E55F954D400390
:10131A00855F4D12060678017988E7B403027805DD
:10132A00C3E55F9840024135C2AF1206301206305B
:10133A00120630D2AF12060B753000E4F531F532E1
:10134A000531E531F470390532789AE67819146076
:10135A0012783214600D787D14600878FA146003EC
:10136A00753200C3E53298401715327531B4789951
:10137A008676C2AF120630D2AF7898867612060603
:10138A001205FCE52A7005307402213378012074B5
:10139A00027806C3E55F9840A77888E6C39403609D
:1013AA0003120606E52A7003021133C2AF120F2B8D
:1013BA00E4F522F523F524F525F526F56AD2AF786A
:1013CA0085E6C333F568E4F545F546F547F548F58E
:1013DA0049F573F52CF52DF53775730875BB1012A1
:1013EA0005F21208AFE5E820ECFBA8BDA9BEE9703A
:1013FA0001F888741208B375730875BB107887E60C
:10140A00FE7602120FA97887EEF6C2AF7564FF1254
:10141A00092B852264852265852266D2AF75220151
:10142A0075240175250175260185636C756D017535
:10143A00B69075A903757D017888E6B40307C27D65
:10144A00307602D27DD268D269753300120E9112BB
:10145A000EB612094B12095212094B1209521209FD
:0E146A004B02147BC2AF120FA9D2AF757300F4
:1014780075BB09120BE41206FB120D0F120D59125F
:101488000952120BD3306D031206FC2067031208B1
:101498004E306703120895120D0F120D7E12095275
:1014A800120BE4306D03120738120D0F120DF512EE
:1014B8000952120BD3306D03120796120D0F120E3C
:1014C8001A120952120BE4306D031207F3120D0FB2
:1014D800120E911209521208AF120BD3120D0F12ED
:1014E8000EB61208B3120952306932206B2F856785
:1014F8006485676585636C756D0179187A0CC3E539
:101508003399400CC269D26A8A357564FF02152581
:10151800C3E55F9401400302147B0215A2306A1BE5
:10152800206B18E535147004C26A816EF535C3E581
:101538005F9401400302147B0215A2753600C3E5CF
:10154800627882985054307404E52A604D7888E6B1
:10155800B40317207D05207607A172307602A172A8
:10156800206B07D26B85676481BA78F0306B05858C
:1015780067647820C3E541985002817B306B1BC2B9
:101588006BC27D307602D27DD26A7535128567646A
:10159800817B0536E55F6002A1A5753600C2AF12F2
:1015A8000F2B7887E6FE7602120FA97887EEF6E40D
:1015B800F522F523F524F525F526F568C26875A901
:1015C8000075B680757D00D2AF1205F2120F2B3070
:1015D8007409C3E5369405400221336145901A0D1C
:1015E8007820121669E520B45A0CA3121669E52072
:1015F800B4A503021607120F4012162702162690EA
:101608001A0378807B0A121669A308DBF9901A0F6F
:10161800788C7B18121669A308DBF9901A2722C266
:10162800AF1216A8121682901A00740E12166EA324
:10163800740412166EA3741412166E901A0378802E
:101648007B0A12166DA308DBF9901A0F788C7B18A9
:1016580012166DA308DBF91216BB121699901A27F9
:1016680022E493F622E6438F01538FFD75EF02754E
:10167800B7A575B7F1F0538FFE22438F02438F0150
:1016880075EF0275B7A575B7F1901A0DF0538FFC79
:1016980022901A0D745AD16E901A0E74A5D16E222A
:1016A8007A3079D07820901A40D169E520F709A3DB
:1016B800DAF7227A3079D0901A40E7D16E09A3DAA6
:1016C800F922AB77A878BB01027984BB020279853D
:1016D800BB03027986BB04027992BB05027987BBFA
:1016E800060279A3BB0702799CBB08027988BB096B
:1016F800027989E8F7227C0512060BDCFB22C2AFCF
:1017080012061B1206221206291206301205FC12B6
:10171800061B1206221206291206301205FC1206B2
:101728001B120622120629120630D2AF22C2AF12AD
:10173800063012062912062212061B1205FC120692
:101748003012062912062212061B1205FC12063058
:1017580012062912062212061BD2AF22AE77AF78E4
:10176800C2AF12061B12061B12061B1205FCDEF284
:101778001206301205FCDFF8D2AF22F106D1FED1F5
:10178800FE757701757801757900F1647C05AD5FA8
:1017980012060BC3ED955F70F5C3E55F9401400A2F
:1017A800C3E55F94FF40320217BFD1CAD127F106C3
:1017B800C2AF75EF12D1FEDCD50579C3E579940384
:1017C800500280C6D1FE0578E5771490009F93F803
:1017D80008C3E57898500280AED1FED1FE0577C3E4
:1017E800E577940A5002809C120F40D127C2AF754A
:0417F800EF12D1FE1D
:0319FD0002108F46
:101A00000E0414FFFFFFFF0304090301015AA5019F
:101A1000FFFFFFFFFF03FFFFFF25D0FAFA04FF01DE
:081A2000007AFF01010003FF41
:101A400023506C6174696E756D50726F3330412331
:101A500023424C48454C492346333930232020202B
:101A60002020202020202020202020202020202076
:101C0000C2AFC2D353D9BF7581C043B20343FF8073
:101C1000752438752503B1C975EF0275E24043F1AB
:101C20002053A4DF75D400D2857DFA780379E67C51
:101C300010752200752300901DD67B0675249875BB
:101C400025013085028142208508D8FBD9F9DCF7CF
:101C500081B4308508D8FBD9F9DCF781B4B189E4C7
:101C600093A3C39A6004DDC381B4DBDBB17B600264
:101C7000812B7B08E493FAA3B15CDBF87A30B15C8A
:101C8000752200752300B17BEAFCEBFDC3ED94FEE9
:101C9000400EB17B8A278B28ED30E0048A828B834B
:101CA000B17B7AC270D8C3ED94FE601350CEBD00F4
:101CB00025EC60097520007521FF0200008100A855
:101CC00027A9280809D804D90281D3B17FEA89AAB3
:101CD000F281C50D81A0C3ED94035049EDA2E092BD
:101CE000007AC5C3E5829400E583941C50902000DF
:101CF00010438F02438F0175B7A575B7F1F030001F
:101D00001FA827A9280809438F01538FFDD804D99C
:101D100002A12089AAE275B7A575B7F1F0A3A10DBC
:101D2000538FFC817C7AC1BD030CE493A3FAB140CC
:101D3000DCF8B138817C817EAA22AB23B15CEBFA5E
:101D4000EA6222752608C3E52313F523E52213F57D
:101D50002250066323A0632201D526EAB1C9B1C986
:101D600075260AEAF4200102D285300102C285B14B
:101D7000C9C3134002C201D526EB22B17FEAFB2082
:101D80008502A17F308502A184752608AE24AF2587
:101D9000C3EF13FFEE13FEB1CDB1C9C3EA13308513
:101DA000024480FA30E703632201C3E52313F523DD
:101DB000E52213F52250066323A0632201D526D91C
:101DC000E52265236523F52222AE24AF250E0FDE22
:101DD000FEDFFCD20122424C48656C693437316326
:041DE000F390060175
:00000001FF
